:1011000012010002000000400516408000000102AC
:1011100000010A06000200000040010009022E0042
:1011200001010080320904000004FF0000000705EF
:101130000202000200070504020002000705860201
:101140000002000705880200020009022E000101CA
:101150000080320904000004FF00000007050202BD
:101160004000000705040240000007058602400019
:101170000007058802400000040309040C03410035
:101180004300430045005300240355005300420030
:101190002D0041004900310036002D00310036009D
:0E11A000410000000000000000000000000000
:100B30005553422D414931362D3136005553422D02
:100B4000414931322D3136005553422D414931361C
:100B50002D36344D005553422D414931322D363416
:100B60004D005553422D414931362D333241005508
:100B700053422D414931362D333245005553422DD4
:100B8000414931322D333241005553422D414931D3
:100B9000322D3332005553422D414931322D3332FB
:100BA00045005553422D414931362D3634410055CB
:100BB00053422D414931362D363445005553422D8F
:100BC000414931322D363441005553422D4149318E
:100BD000322D3634005553422D414931322D3634B1
:100BE00045005553422D414931362D393641005586
:100BF00053422D414931362D393645005553422D4A
:100C0000414931322D393641005553422D41493148
:100C1000322D3936005553422D414931322D393666
:100C200045005553422D414931362D31323841006E
:100C30005553422D414931362D31323845005553F7
:100C4000422D414931322D31323841005553422D28
:100C5000414931322D313238005553422D4149310D
:100C6000322D31323845005553422D41492D4F54D4
:040C700048455200A1
:100D7C00C104020C00004228AC00004128AB000268
:0C0D8C00100000010E000114FF010FFE1A
:100E4F00E490E68AF090E6BEE090E68BF022E49024
:100E5F00E68BF090E6BBE0FF90E6BAE075F008A4F1
:100E6F00222FFFEC35F0FEE42FF58274503EF58310
:100E7F002290E740F0E490E68AF090E68B2225334B
:100E8F00F533E5363532F532C3E5359537F535E5CA
:100E9F00349536F534227586005391EF90E65D2236
:100EAF0074402539F582E434E7F58322C3E539959B
:100EBF0037E538953622AD377AE779407F40AB0773
:100ECF00222403F582E5F0345022E5332539F582EB
:100EDF00E5323538F58322E0FD90E6BBE0C413130D
:100EEF00540322F582E43428F58322854782854610
:100EFF0083A37402F022854982854883A37407F087
:080F0F00227BFF7A0B793C22E2
:0417DC004380022222
:0417E0005380FD2213
:0417E40063800222FA
:1012D900E490E671F090E672F075B3FF75B4FF75AE
:1012E900B5FF75B6FFFEFD7801AF06EF0880010373
:1012F900D8FDF5B18EB08DA08D9090401BEDF00D0D
:10130900ED70E40EEE70E0F5B3F5B5FEFD7801AFD2
:1013190006EF08800103D8FDF5B18DA090401C743B
:1013290001F0AF90ACB0E4F0EFB50504EC6E6003EA
:10133900750F010DED70D60EEE70D2E50FB4FE03F8
:09134900E4F50FE4F5B4F5B62259
:1013BB008B318A328933E4F53412179B8F35E5353F
:1013CB0025E02402901188F0E4F534AF35EF339526
:1013DB00E0FEC3E5349FEE6480F87480985027AB31
:1013EB0031AA32A9338534827583001211AEFDE523
:1013FB003475F002A4248AF9741135F08982F583CF
:07140B00EDF0053480C5225D
:100647001217D490E678E05410C4540F4450F50BB9
:1006570013E433F516120EC77D017F037E001210D7
:10066700B890E740E0541FF514444090110AF0E5B4
:1006770014541FB41E0040030207BF900689F828D0
:1006870028730206E30206E50206EE0206F40206F6
:10069700FA020700020709020712020712020712ED
:1006A70002071B02072402072D02073602073F0233
:1006B700074702074F02075702075F02076702074C
:1006C7006F02077702077F02078702078F020797E4
:1006D70002079F0207A70207AF0207B780007BFF49
:1006E7007A0B79300207C5120F100207C5120F10D7
:1006F7000207C5120F100207C57BFF7A0B79480264
:1007070007C57BFF7A0B79480207C57BFF7A0B7910
:10071700550207C57BFF7A0B79620207C57BFF7A13
:100727000B796F0207C57BFF7A0B797C0207C57BC4
:10073700FF7A0B79890207C57BFF7A0B7995807E53
:100747007BFF7A0B79A280767BFF7A0B79AF806E7D
:100757007BFF7A0B79BC80667BFF7A0B79C9805E59
:100767007BFF7A0B79D580567BFF7A0B79E2804E37
:100777007BFF7A0B79EF80467BFF7A0B79FC803E13
:100787007BFF7A0C790980367BFF7A0C7915802EEE
:100797007BFF7A0C792280267BFF7A0C7930801ECA
:1007A7007BFF7A0C793E80167BFF7A0C794C800EA2
:1007B7007BFF7A0C795980067BFF7A0C79671213D5
:1007C700BB1212D990E61074A0F090E611F0000069
:1007D7000090E612F0000000E490E613F00000003D
:1007E70090E61474E0F0000000E490E615F090E65F
:1007F700047480F00000007402F00000007406F03A
:10080700000000E4F000000090E618F0000000741B
:1008170011F000000090E61A7409F000000043AFE1
:1008270001120F1743B67F43B202D2001217DC1230
:0508370017E40217E0C8
:10141200E5BB30E72D00000090E6AFE0FE90E6B0BD
:10142200E07C002400F50DEC3EF50CD3E50D9400B4
:10143200E50C9400400CE50C9402500690E64874CA
:1014420006F0E58070047F0180027F00EF90E68065
:0D14520030E005E04408F022E054F7F022FD
:0217EC00D32206
:0217EE00D32204
:0217F000D32202
:1014A50090E680E030E71800000090E6247402F032
:1014B500000000E490E625F0000000D2048016004C
:1014C5000000E490E624F000000090E6257440F06A
:0D14D500000000C20490E6BAE0F515D32235
:0917BA00E515120E8004F0D322A3
:0817CC0090E6BAE0F50AD32211
:0917C300E50A120E8004F0D322A5
:0217F200D32200
:0217F400D322FE
:0217F600D322FC
:10008000E4F53AF53B90E6B9E012120E0198100142
:10009000A41101BB1201232001562101632301E8B1
:1000A0003501E23802F3910543A20543A3053DA9BA
:1000B000051CAC00D5B40303BA0326BB0424BC0260
:1000C0001DBE02D2BF0200D0020BD1046FD200E9E4
:1000D000D400000643E5BBF45480FF90E6F4E054FE
:1000E000044F90E740F002031E90E6B8E020E71EC0
:1000F000120E4F90E6A0E020E1F990E740E0FF907B
:10010000E6BAE0FEE42EF582E4344002015C90E6BB
:10011000BAE0FFE42FF582E43440F583E090E74055
:100120000201B390E6BBE0C4333354C0120E661232
:100130000ED0F583EFF0120E67FFA3E07C00120EE5
:1001400070E090E740F0120E67FFA3E0120E70E03F
:1001500090E741020516120E5D120ED0F583EFF006
:10016000020645120E5D120ED0F583EFF090E6BC4C
:10017000120EE67A005403FB120E672BFFEA120EF2
:1001800073EDF090E6BD120EE6FB120E672BFFEA50
:10019000120E73EDF0020645120E4F90E6A0E0201D
:1001A000E1F9802B904015E090E740F0904016E098
:1001B00090E741F0E490E68A020516120E4F90E6B1
:1001C000A0E020E1F990E742E05403904014F09061
:1001D000E740E0904015F090E741E0904016F002D3
:1001E000064590E6F574FFF090E6997480F0000003
:1001F00000F0000000F0000000F000000002031E0C
:1002000090E604E0F531433180800990E604E0F5A2
:100210003153317F000000E531F0020645120E4FE8
:1002200090E6A0E020E1F990E740E0904000F090F7
:10023000E741E0904001F090E742E0904002F0900A
:10024000E743E0904003F090E744E0904004F090F2
:10025000E745E0904005F090E746E0904006F090DA
:10026000E747E0904007F090E748E0904008F090C2
:10027000E749E0904009F090E74AE090400AF090AA
:10028000E74BE090400BF090E74CE090400CF09092
:10029000E74DE090400DF090E74EE090400EF0907A
:1002A000E74FE090400FF090E750E0904010F09062
:1002B000E751E0904011F090E752E0904012F0904A
:1002C000E753E0904013F090E754E090401DF002B7
:1002D0000645904019E4F01216B8904017E090E7F8
:1002E00040F0904018E090E741F090E68B7402F007
:1002F00002064590E740E50FF090E6BFE090E68A01
:1003000002051690401AE05407F5146003B4020881
:1003100090E74074BBF0800690E740E514F0120EC1
:100320008404F002064590401AE05407F514600773
:100330006402600302041C90E74074BBF090E6BBCB
:10034000E0C313FFE5B154802FF5B1E090E6C4F0AF
:1003500090E6BAE090E6C5F090E6C4E0700990E659
:10036000C5E070031217E090E6BDE0FE90E6BCE049
:100370007C002400F513EC3EF512E51345127003E2
:10038000020460E5BB30E7F2E5AB20E1ED30042389
:10039000D3E5139400E5129402403F90E6D0740236
:1003A000F0000000E490E6D1F0000000750802F5CE
:1003B00009803ED3E5139440E5129400E440179081
:1003C000E6D0F000000090E6D17440F00000007527
:1003D0000800F509801B90E6CFF0E51290E6D0F01A
:1003E000000000E51390E6D1F0000000851208F54A
:1003F00009E4F5BB000000E5BB30E7FB000000C3EB
:10040000E5139509F513E5129508F512E5B1547F4A
:1004100004FFE5B154802FF5B102037A90E740E57F
:1004200014F0803CE5BB30E737E5AC20E03290E6E5
:10043000BBE090E6CEF000000090E6BAE090E6CF98
:10044000F000000090E6BDE090E6D0F000000090E3
:10045000E6BCE090E6D1F000000075BB06000000AD
:10046000120E8404F090E6A0E04480F0020645906D
:100470004000E090E740F0904001E090E741F090CC
:100480004002E090E742F0904003E090E743F090B4
:100490004004E090E744F0904005E090E745F0909C
:1004A0004006E090E746F0904007E090E747F09084
:1004B0004008E090E748F0904009E090E749F0906C
:1004C000400AE090E74AF090400BE090E74BF09054
:1004D000400CE090E74CF090400DE090E74DF0903C
:1004E000400EE090E74EF090400FE090E74FF09024
:1004F0004010E090E750F0904011E090E751F0900C
:100500004012E090E752F0904013E090E753F090F3
:10051000401DE090E754120E5302064590E6B5E008
:1005200054FEF090E6BFE0120E5090E6BBE090E67D
:10053000B3F090E6BAE090E6B4F002064575160115
:10054000430B0190E6BAE0753200F533A3E0FEEE0E
:10055000423290E6BEE0753400F535A3E0FEEE428F
:100560003490E6B8E064C060030205EAE53545343E
:10057000700302064590E6A0E020E1F9C3E535945A
:1005800040E534940050088534368535378006754B
:10059000360075374090E6B9E0B4A31EE4F538F5AF
:1005A00039120EBB5038120ED9E0FF120EAFEFF029
:1005B0000539E53970EB053880E7E4F538F539128F
:1005C0000EBB5010120EAF74CDF00539E53970EF47
:1005D000053880EB120EC5AF33AE321210B8120ED2
:1005E00084E537F0120E8D02056C90E6B8E06440A9
:1005F0007053E5354534604D120E84F090E6A0E06E
:1006000020E1F990E68BE0753600F53790E6B9E029
:10061000B4A31EE4F538F539120EBB501E120EAF0E
:10062000E0FF120ED9EFF00539E53970EB0538809F
:10063000E7120EC5AF33AE3212158EE537120E8DAE
:070640000205F2D322C322E0
:1016DD00C0E0C083C082C085C084C086758600D23C
:1016ED0001120EA87401F0D086D084D085D082D09E
:0416FD0083D0E03284
:10172500C0E0C083C082C085C084C086120EA57487
:0F17350004F0D086D084D085D082D083D0E0322B
:10174400C0E0C083C082C085C084C086120EA57468
:0F17540002F0D086D084D085D082D083D0E0320E
:1015C300C0E0C083C082C085C084C08675860085A4
:1015D3004A46854B47120EFA854248854349120F06
:1015E30005120EA87410F0D086D084D085D082D096
:0415F30083D0E0328F
:10170100C0E0C083C082C085C084C086758600D217
:1017110003120EA87408F0D086D084D085D082D070
:0417210083D0E0325F
:1014E200C0E0C083C082C085C084C086758600907B
:1014F200E680E030E712854246854347120EFA85C0
:101502004A48854B49120F05120EA87420F0D08666
:0B151200D084D085D082D083D0E0329E
:010FFF0032BF
:0117F80032BE
:0117F90032BD
:0117FA0032BC
:0117FB0032BB
:0117FC0032BA
:0117FD0032B9
:0117FE0032B8
:0117FF0032B7
:0118000032B5
:0118010032B4
:0118020032B3
:0118030032B2
:0118040032B1
:0118050032B0
:0118060032AF
:0118070032AE
:0118080032AD
:0118090032AC
:01180A0032AB
:01180B0032AA
:01180C0032A9
:01180D0032A8
:01180E0032A7
:01180F0032A6
:0118100032A5
:0118110032A4
:0118120032A3
:0118130032A2
:0118140032A1
:0118150032A0
:01181600329F
:01181700329E
:01181800329D
:01181900329C
:01181A00329B
:10151D00AB07AA06AC05E4FDE516600B7E000DEEEB
:10152D0024AE120EF2EAF0AE050D74AE2E120EF2CE
:10153D00EBF0AF050D74AE2F120EF2ECF07A287BA6
:0B154D00AEAF0B12177FAF0B0215585A
:10158E008E3C8F3D8D3E8A3F8B40E4F541E541C355
:10159E00953E5020053DE53DAE3C7002053C14FFE6
:1015AE00E5402541F582E4353FF583E0FD12151D3A
:0515BE00054180D92267
:1010B8008E3C8F3D8D3E8A3F8B40E4FDF541E51621
:1010C8006012E53CFF7E000DEE24AEF582E4342884
:1010D800F583EFF0AE050D74AE2EF582E43428F5F5
:1010E80083E53DF07A287BAEAF0B12177FAB40AAA1
:0810F8003FAD3EAF0B02176390
:03004300021000A8
:0300530002100098
:101000000216DD0002174400021725000217010036
:101010000215C3000214E200020FFF000217F800DD
:101020000217F9000217FA000217FB000217FC0072
:101030000217FD000217FE000217FF000218000051
:10104000021801000217F80002180200021803003B
:101050000218040002180500021806000218070012
:10106000021808000217F8000217F8000217F8002B
:101070000218090002180A0002180B0002180C00DE
:1010800002180D0002180E0002180F0002181000BE
:10109000021811000218120002181300021814009E
:1010A000021815000218160002181700021818007E
:0810B0000218190002181A00D1
:1016B8007400F58690FDA57C05A3E582458370F945
:0116C80022FF
:0817D400E4F51CD2E9D2AF22BA
:1015580090E678E020E6F9C2E990E678E04480F089
:10156800EF25E090E679F090E678E030E0F990E653
:1015780078E04440F090E678E020E6F990E678E0FC
:0615880030E1D6D2E92299
:10162B00A90790E678E020E6F9E51C702390E678B0
:10163B00E04480F0E925E090E679F08D17AF03A93F
:10164B00077518018A19891AE4F51B751C01D32239
:02165B00C322A8
:1015F700A90790E678E020E6F9E51C702590E678E3
:10160700E04480F0E925E0440190E679F08D17AFDA
:1016170003A9077518018A19891AE4F51B751C03B4
:04162700D322C322E5
:03004B00020C7430
:100C7400C0E0C083C082C085C084C086758600C0C1
:100C8400D075D000C000C001C002C003C006C007B8
:100C940090E678E030E206751C06020D5E90E67878
:100CA400E020E10CE51C64026006751C07020D5E81
:100CB400E51C24FE605F14603624FE7003020D4FB1
:100CC40024FC7003020D5B24086003020D5EAB1864
:100CD400AA19A91AAF1B051B8F827583001211AEC6
:100CE40090E679F0E51B65177070751C05806B90B4
:100CF400E679E0AB18AA19A91AAE1B8E8275830097
:100D04001211DB751C02E5176401704E90E678E061
:100D14004420F08045E51724FEB51B0790E678E0F3
:100D24004420F0E51714B51B0A90E678E04440F03F
:100D3400751C0090E679E0AB18AA19A91AAE1B8EAF
:100D4400827583001211DB051B800F90E678E04466
:100D540040F0751C008003751C005391DFD007D050
:100D640006D003D002D001D000D0D0D086D084D019
:080D740085D082D083D0E0326B
:101763001215F7E51C24FA600E146006240770F3C3
:0C177300D322E4F51CD322E4F51CD322A1
:10177F0012162BE51C24FA600E146006240770F372
:0C178F00D322E4F51CD322E4F51CD32285
:100D980060802800013F01010101010700030202F0
:100DA80002020200F5F7F7F7F7F7F7F7000000007F
:100DB8000000003F013F0101010101070205000099
:100DC80000000000F6F7F7F7F7F7F7F70000000064
:100DD8000000003F01100138010101070001000B6C
:100DE80002020200F3F7F5F7F7F7F7F70000006ED5
:100DF8000000003F0138010101010107020D000058
:100E080000000000F6F7F7F7F7F7F7F7002D0000F6
:100E18000000003F60242887000000000000000058
:100E280000000000000000000000000000000000BA
:100E3800000000000000000000000000472880E0DB
:060E48008000F7EA4E00F5
:100F170090E60174EAF090E6F574FFF0902880E01F
:100F270090E6F3F0902881E090E6C3F0902882E005
:100F370090E6C1F0902883E090E6C2F0902885E023
:100F470090E6C0F0902886E090E6F4F075AF07745D
:100F570028F59A7400F59B759DE4E4F59EFF90E6ED
:100F67007BE090E67CF00FBF80F490E67174FFF0B1
:100F7700F5B490E672E04480F043B680000000E4E8
:100F870090E6C4F000000090E6C5F0902887E09056
:100F9700E6C6F0902888E090E6C7F0902889E090B0
:100FA700E6C8F090288AE090E6C9F090288BE09098
:100FB700E6CAF090288CE090E6CBF090288DE09080
:0C0FC700E6CCF090288EE090E6CDF02201
:0A17B0000001020203030404050512
:10135200EC4EFEED4F24B0F58274173EF583E49314
:10136200FF3395E0FEEF24A1FFEE34E68F82F58392
:101372002290E6BCE0547EFF7E00E0D394807C00A5
:1013820022F0E5242401F524E43523F523E4352273
:10139200F522E43521F52122AF28AE27AD26AC2572
:1013A200AB24AA23A922A821C30211FDE52E2524DC
:0913B200F582E52D3523F58322B7
:1009E500E4F52CF52BF52AF529C203C200C202C293
:1009F500011206477E117F008E448F45754C117597
:100A05004D1275421175431C754A11754B4A754E49
:100A150011754F78EE54E07003020AD1752D0075FB
:100A25002E808E2F8F30C374AC9FFF74119ECF2400
:100A350002CF3400FEE48F288E27F526F525F52410
:100A4500F523F522F52112139A500A1213AE74CD2F
:100A550012138380F1E4F524F523F522F521121311
:100A65009A5017E5302524F582E52F3523F583E0E7
:100A7500FF1213AEEF12138380E4852D44852E45B6
:100A850074002480FF741134FFFEC3E54D9FF54DBE
:100A9500E54C9EF54CC3E5479FF547E5469EF54673
:100AA500C3E5499FF549E5489EF548C3E5439FF5EC
:100AB50043E5429EF542C3E54B9FF54BE54A9EF55E
:100AC5004AC3E54F9FF54FE54E9EF54ED2E843D814
:100AD5002090E668E04409F090E65CE0443DF0D201
:100AE500AFD20512165D90E680E054F7F0538EF80C
:100AF500C20330010512083CC2013003291217EC6C
:100B05005024C2031216C920001690E682E030E791
:100B150004E020E1EF90E682E030E604E020E0E446
:0B0B2500120FD31217EE12141280C73B
:10083C0090E6B9E070030208ED147003020941243C
:10084C00FE700302099B24FB70030208E71470037B
:10085C000208E1146073146076240560030209D168
:10086C001217F040030209DD90E6BBE024FE602283
:10087C0014603324FD601114602224067048E54492
:10088C0090E6B3F0E5458037E54C90E6B3F0E54DE6
:10089C00802DE54690E6B3F0E5478023E54890E6E9
:1008AC00B3F0E549801990E6BAE0FF12168CAA065F
:1008BC00A9077B01EA494B600DEE90E6B3F0EF908F
:1008CC00E6B4F00209DD0209D61217C30209DD12E3
:1008DC0017CC0209DD1214A50209DD1217BA0209A0
:1008EC00DD1217F240030209DD90E6B8E0247F60C8
:1008FC00151460192402703AA200E43325E0FFA21B
:10090C0002E4334F8018E490E740F0801612137322
:10091C0040047D0180027D00121352E0540190E7E7
:10092C0040F0E4A3F090E68AF090E68B7402F002BB
:10093C0009DD0209D61217F440030209DD90E6B86E
:10094C00E024FE6016240260030209DD90E6BAE0A2
:10095C00B40105C2000209DD0209D690E6BAE070C6
:10096C002C12137340047D0180027D00121352E09F
:10097C0054FEF090E6BCE05480131313541FFFE0B8
:10098C00540F2F90E683F0E04420F08044803B121B
:10099C0017F6503D90E6B8E024FE60192402703141
:1009AC0090E6BAE0B40104D200802690E6BAE06486
:1009BC0002601E801512137340047D0180027D00BD
:1009CC001213528008120080500790E6A0E04401F8
:0909DC00F090E6A0E04480F02256
:030033000217E8C9
:0417E80053D8EF32B1
:100FD30090E682E030E004E020E60B90E682E03029
:100FE300E119E030E71590E680E04401F07F147EDC
:0C0FF3000012145F90E680E054FEF02233
:1016C90090E682E044C0F090E681F0438701000093
:0416D90000000022EB
:10165D0030050990E680E0440AF0800790E680E0CE
:10166D004408F07FDC7E0512145F90E65D74FFF098
:0F167D0090E65FF05391EF90E680E054F7F02293
:02168C00A907AC
:10168E00AE4EAF4F8F828E83A3E064037017AD0111
:10169E0019ED7001228F828E83E07C002FFDEC3ECF
:0916AE00FEAF0580DF7E007F0025
:0116B7002210
:10145F008E318F3290E600E054187012E53224017D
:10146F00FFE43531C313F531EF13F532801590E6F4
:10147F0000E05418FFBF100BE53225E0F532E531DF
:10148F0033F531E5321532AE31700215314E60054C
:06149F001216B880EE22D7
:0300000002124D9C
:0C124D00787FE4F6D8FD75814F02129402
:1011AE00BB010CE58229F582E5833AF583E02250F6
:1011BE0006E92582F8E622BBFE06E92582F8E22240
:0D11CE00E58229F582E5833AF583E493225A
:1011DB00F8BB010DE58229F582E5833AF583E8F04A
:1011EB00225006E92582C8F622BBFE05E92582C8F6
:0211FB00F222DE
:1011FD00EB9FF5F0EA9E42F0E99D42F0E89C45F048
:01120D0022BE
:10120E00D083D082F8E4937012740193700DA3A36F
:10121E0093F8740193F5828883E473740293686083
:06122E00EFA3A3A380DF83
:10179B00E4FFFE121234600C0FEF70010E09E970BA
:0517AB00F20A80EF22AC
:101259000209E5E493A3F8E493A34003F68001F2BD
:1012690008DFF48029E493A3F85407240CC8C33396
:10127900C4540F4420C8834004F456800146F6DF65
:10128900E4800B0102040810204080900D7CE47E6C
:10129900019360BCA3FF543F30E509541FFEE4935A
:1012A900A360010ECF54C025E060A840B8E493A321
:1012B900FAE493A3F8E493A3C8C582C8CAC583CA4C
:1012C900F0A3C8C582C8CAC583CADFE9DEE780BE04
:010E4E0000A3
:10123400BB010689828A83E0225002E722BBFE02B8
:09124400E32289828A83E49322EB
:00000001FF
